:020000040000FA
:060000006CEF07F0120096
:020006000000F8
:0600080004EF08F01200F5
:080018000CEF08F08BEF07F07C
:020020001200CC
:0E002200010006000000BA030000020000000A
:100030000001E56BE969EA69EB69E86B010EEC6FB9
:1000400012000001E5511EE1040108BF93D1000137
:10005000400EFE6F0001A10EFC6F000EFD6F2DEC37
:1000600006F00001010EE56FED6B400EED5D01E362
:1000700081D1ED51EA6A600FE96E000EEA22EF6A63
:10008000ED2BF3D70001A151080A01E170D1040A58
:1000900001E131D1050A01E12CD10E0A01E1F5D0CF
:1000A000010A01E1ECD0030A01E194D0010A4CE01D
:1000B000070A40E0010A01E05BD10001020E606F17
:1000C0003A0E616F010E626F636F646B100E656FA5
:1000D000666B676B686B700E696F6A6B6B6B030E98
:1000E0006C6F6D6B6E6B300E6F6F706B0E0E716F91
:1000F000726B736B746B040E756F766B776B200E7F
:10010000786F796B080E7A6F7B6B7C6B7D6B020E60
:100110007E6F7F6B806BF00E816F826B836B010E45
:10012000846F856B866B8769A50E996F04010CBF80
:1001300021D1DCD00001010EEC6F0001A25101E0E1
:1001400013D10001EC6B10D1400E0001E66FE76B9C
:10015000000EE65D020EE7591FE22FDAE6C000F05E
:10016000E7C001F0026A060E1F0BE6C0F6FFE7C00B
:10017000F7FF02C0F8FF06E0D890F636F736F836FB
:10018000E806FAE1940EA66E24DA72EC06F000019D
:10019000E62B000EE723DCD7ED6BEDC0A9FFA868C6
:1001A000040EA66E72EC06F014DA0001ED51ED2B90
:1001B000006E016A026AFF0E005C000E0158000E1C
:1001C0000258EBE3F66AF76A200EF86E940EA66EFC
:1001D00000DACAD0300EA45D06E10001EC5101E066
:1001E000C3D092D9C1D0F00EA45D02E1B3D9BCD086
:1001F000E8680001E9190CE1E868EA1909E1E86832
:10020000EB1906E1A2C0E9F0A3C0EAF0A4C0EBF04C
:10021000E90EE96E000EEA6EEE500001A21901E04F
:10022000A3D0EE50A31901E09FD0EE50A41901E035
:100230009BD001E099D00001ED6B0001A6510001B7
:10024000ED5D01E391D0BDD9A70FE96E000EEA2262
:10025000EF50E66EE851EA6A600FE96E030EEA229B
:10026000E552E750EF6EE82BE92B000EEA23EB2373
:10027000200EE85D01E1E4D80001ED2BDED7E0D8E7
:100280000001E969EA69EB6970D00001070E606F4F
:10029000A2C061F0A3C062F0A4C063F0A5C064F086
:1002A000A6C065F0A2C0F6FFA3C0F7FFA4C0F8FF88
:1002B0000001ED6B0001A6510001ED5D14E2F00EAE
:1002C0000001A45D0AE1A2510001ED25A96EA66A14
:1002D000A68084D9A8CFEFFF04D071D97FD9F5CFFC
:1002E000EFFFED2BE7D704010CBF44D00001400E17
:1002F00033D041D839D000010C0E606F010E616F10
:10030000626F160EF66E100EF76E0900F5CF63F0F1
:100310000A00F5CF64F0060E656F100E666F676B0E
:10032000686B0D0E696F600E6A6F400E6B6F6C6BC1
:100330006D6B6E6B6F69706971697269736B7469EB
:100340007569766B7769786979697A697B697C699F
:1003500004010CBF0FD00001FA6F0001600EF86FAE
:10036000000EF96F07EC06F00001E56B120050D8A3
:100370000001E56B1200F66A100EF76EF86A0001D4
:10038000EE6B400E0001EE5D0DE209000001EE5142
:10039000EA6A600FE96E030EEA22F5CFEFFF000173
:1003A000EE2BEFD703010D0E666F0301600E676F32
:1003B000F66A100EF76EF86A940EA66E0001B50E7E
:1003C000F46FE8D83F0EF66E100EF76EF86A000173
:1003D0003F0EEE6F0001EE51EA6A600FE96E030E08
:1003E000EA22EF50F56E0C000001EE511F0B07E101
:1003F000E4D8A40EA66E0001B50EF46FCBD80A00A7
:100400000001EE5101E103D00001EE07E3D7120035
:1004100004D8FF000000000012000301B869B969A8
:100420000301B8C300F0B9C301F0B807000EB95B0F
:100430000050011004E06D926D6ABFD8F1D7120030
:100440000001F06BE8C000F0016A026A0050000190
:10045000E95DF66E01500001EA59F76E02500001A5
:10046000EB59F86E1F0EF6140001F16FE00EF61650
:100470000001EF6B200E0001EF5D1FE20001F15162
:1004800015E10001E8510FE00001F051EA6A600F48
:10049000E96E030EEA22EF50F56E0D000001F02B1D
:1004A0000001E80702D0F5680D0004D0F5680D00E2
:1004B0000001F1070001EF2BDDD70A00A40EA66EA4
:1004C0000001B50EF46F66D80001EF6B0001E85132
:1004D0000001EF5D18E20001F0510001EF25EA6A2A
:1004E000600FE96E030EEA22EF50E66E0001EF5155
:1004F000EA6A600FE96E030EEA22E552E750EF6EFA
:100500000001EF2BE3D71200A2C0F6FFA3C0F7FF54
:10051000A4C0F8FF0001F26B0001A6510001F25DDA
:1005200018E23A0E0001D880A6550001F225EA6AC9
:10053000A70FE96E000EEA22EF50F56E0C00C40E14
:10054000A66E0001B50EF46F25D809000001F22B4C
:10055000E3D712000001F36B0001A6510001F35D27
:1005600018E20001A2510001F325A96E3A0E000124
:10057000D880A6550001F325EA6AA70FE96E000EA0
:10058000EA22EF50A86E040EA66E23D80001F32BCA
:10059000E3D71200F29EB50E0001F45D05E0030EF4
:1005A000D36E0300FED7FF00550EA76EAA0EA76EEE
:1005B000A682A6B2FED7A69412000400120009007B
:1005C00012003A0E0001D880A6550001ED25EA6A16
:1005D00012000001B50EF46FCAEF02F0F2DF660FF1
:0805E000E96E000EEA22120090
:0805E8006C5033E16896040138
:1005F00000513C0BE842E8420D0829E1180E0219AF
:1006000024E1040E031921E1100E026F040E036FA2
:100610000301A96BA951006E016A080E005C000E6F
:10062000015813E2A951EA6A180FE96E040EEA2292
:10063000EF50E66EA951EA6A100FE96E040EEA2245
:10064000E552E750EF6EA92BE5D70AD8010C3AD84E
:10065000010C040E6C5C03E168964BD8010C000C95
:10066000040104BF046B0301A86BA06BA16BA66B14
:10067000A76B50EC04F00301AA6BAA51006E016A4B
:10068000010E005C000E01581BE2A15119E1AA51B4
:10069000F66EF76AD890F636F736D60EF6260E0EB8
:1006A000F7220900F5CF00F00800F5CF01F004D0E3
:1006B00001C0FAFF0050F96EFBDF0301AA2BDDD762
:1006C000F8EF03F0020E0301A05D0EE178D80401FB
:1006D000180E026F040E036F080E016F00BD02D0EA
:1006E000C80E05D0880E03D0BCD8CBD88C0E006FB6
:1006F0001200040E0301B45D09E112C46EFF6E50D6
:10070000000802E2050E01D0030EB46F0301A0053C
:1007100010E111D8020E0301A85D03E10401840E6B
:1007200006D0040104BD02D0C80E01D0880E046FAB
:10073000120031EF04F00301080EA65D000EA75968
:100740000DE2A6C3ABF3A7C3ACF3A85102E1010EBF
:1007500003D0A80506E1020EA86F03D0080EAB6F08
:10076000AC6B0401049304910301AC510401041324
:10077000ABC305F40301AB51A65DA66FAC51A759FD
:10078000A76F180EA46F040EA56F0301B5A30ED0BA
:100790000301AB51AC1112E0A2C3F6FFA3C3F7FFF4
:1007A0000800F55063D8AB07AC5BF2D70301AB513F
:1007B000AC1104E06ED8AB07AC5BF8D71200030EA7
:1007C000040100150301AE6F01C4ADF3A651AD25C0
:1007D000A66FA751AE21A76F180EA26F040EA36FCC
:1007E000AD51AE1104E055D8AD07AE5BF9D712009C
:1007F0006D980301A15105E144D8840E006F0401F6
:100800001DD0040110AF1CD00301A6510401165DD8
:100810000301A7510401175904E216C4A6F317C433
:10082000A7F389DF0301010EA06F2BD8800E006FA4
:100830000401180E066F040E076FC80E046F120035
:100840000301020EA06F0401056BC80E046F0401C2
:10085000080E016F180E026F040E036FC80E006FB2
:1008600012000301A06B0401046B1200A4C3E9FF92
:10087000A5C3EAFFEF6EA42B000EA523A22BA32392
:1008800012000401080E016F100E026F040E036FB8
:100890001200A2C3E9FFA3C3EAFFEF5036EF04F052
:1008A00004011051600BE842E842E842E842E842A5
:1008B000000901E012001151070A40E00B0A3EE076
:1008C000070A33E0010A23E00B0A1FE0020A1DE0D9
:1008D000030A19E0080A10E0010A0CE00F0A08E018
:1008E000030A01E012000DD90301040EB46F1200D7
:1008F0009FEF04F0D6EF04F004D90301B60EA26F07
:10090000030EA36F0CD0F5EF04F025EF05F0FDD832
:100910000301A26FA36BB70EA227030EA32303014B
:10092000B5930301010EA66F1200EFD8EA6AB70F64
:10093000E96E030EEA2212C4EFFF12001200800ECD
:100940000401105D32E11351030A1FE0010A0AE0BD
:10095000030A29E1D6D80301160EA26F0E0EA36F6B
:10096000120E1ED0B4D8CC0EF6260E0EC2D8020E31
:100970000301F76AA225F66EA351F7220900F5CF0D
:10098000A6F30A00F5CFA7F30ED0A1D8D00EF62615
:100990000E0EAFD8A2C3F6FFA3C3F7FF0800F550B1
:1009A0000301A66FA76B0301B5831200AAD8716A71
:1009B000726A736A746A756A766A776A0301B36FDA
:1009C0000301B70EB16F030EB26FFFEC06F012C455
:1009D000B6F30401125104E10301050EB46F1200D5
:1009E0000301060EB46FF2EF05F00401186B196BEA
:1009F000040110511F0B020A0DE0030A09E0010A6D
:100A000016E17FD80301B5A112D0040118830FD0DD
:100A100078D80DD050D801E0010E62D8A4C3E9FF08
:100A2000EA6EEF50040B03E00401010E186F03019E
:100A3000A1050AE10301180EA26F040EA36F0301C2
:100A4000B5930301020EA66F1200040112050EE118
:100A500010511F0B00090AE154D8030E0401115D67
:100A600003E10301B58102D00301B59104011251E4
:100A700021E110511F0B02081DE114510F0B000959
:100A800019E019D801E0010E2BD8030E0401115D05
:100A900002E1840E03D014AF07D0400EA4C3E9FFD7
:100AA000A5C3EAFFEF6E1200880EA4C3E9FFA5C339
:100AB000EAFFEF6E120029D80F0B080DF350016A00
:100AC000000F006E040E01221451800B120019D881
:100AD00004011251F66EF76AD890F636F736120016
:100AE000040DF35003010024A46F000E0120A56F34
:100AF0001200F7220900F5CFA2F30A00F5CFA3F305
:100B000012000301010EA16F1200FBDF040114515A
:020B10001200D1
:0E0B1200040110511F0B010801E012001451E4
:100B200001E01200060E115D24E11351230A1FE0BB
:100B3000010A0DE0030A1BE1BDD80301B60505E17A
:100B400003013A0EA26F0E0EA36F090E0DD0B2D89C
:100B50000301B60505E10301AF0EA26F0E0EA36FF0
:100B60000301B60504E11D0E0301A66FA76B030187
:100B7000B58304011051600BE842E842E842E842C4
:100B8000E842010801E0120011510B0A25E0080AB1
:100B900017E0090A11E0080A09E00B0A05E0080A53
:100BA00001E01200F0EF05F0F1EF05F083D803014A
:100BB000F50EA26F000E09D07DD813C4F5F0120017
:100BC00079D80301F60EA26F000EA36F0301B5934F
:100BD0000301010EA66F12006DD812C4F6F01200C8
:100BE000120012000001F76B1E0E716E0401400E20
:100BF000096F200E0A6F040E0B6F880E086F040138
:100C0000600E0E6F040E0F6F400E0C6F120000018D
:100C1000FA51400802E2400EFA6FFB6BFA51FB5D9D
:100C200013E2FB51EA6AF825E96EF951EA22EF5026
:100C3000E66EFB51EA6A600FE96E040EEA22E552A5
:100C4000E750EF6EFB2BEAD7FAC00DF4400E04011B
:100C50000C170C7D880E0C1312000001F76B0401B9
:100C600008BF25D009510001D880FE5502E209C411
:100C7000FEF0F76BFE51F75D13E2F751EA6A200FC1
:100C8000E96E040EEA22EF50E66EF751EA6AFC259F
:100C9000E96EFD51EA22E552E750EF6EF72BEAD7F5
:100CA0000401400E096F0817087D880E0813000123
:0C0CB000F75112000301020EA16F1200A8
:040CBC006DB606D03B
:100CC0006D6A696A6D860301010EB46F0301B40594
:100CD00008E16DBA06D0686A696A69806988020E9F
:100CE000B46F12000301B45101E1120068B446D898
:100CF0006DB2120068B059D868B817D868BA45D82C
:100D0000030E0301B45D01E212000301AF6B040E98
:100D1000AF5D0AE268A608D0F4EC02F0000901E138
:100D200068960301AF2BF3D7120069CFB0F3040E1E
:100D3000696E68986D828C90A19AA08A0300A15078
:100D4000200B05E1D050080B02E10300F8D7A09A70
:100D50000301B05169120301D50EB86F020EB96FCD
:100D60000301B8C300F0B9C301F0B807000EB95BC6
:100D70000050011002E00400F3D712006D92699454
:100D800068A402D06894FCD7120070A00CD0800E2A
:100D90000401005D07E1840E0401045D03E1040128
:100DA0008C0E006F7090689A12006A6A686A9F0ED3
:100DB0006B6E7B0E696E6E6A716A726A736A746AB0
:100DC000756A766A776A160E706E68A604D06896A1
:100DD000DDEC02F0FAD76D9831EC04F00401080E56
:100DE000016F100E026F040E036F8C0E006F030173
:100DF000B5910301B66B0301030EB46F1200B1C3CA
:100E0000E9FFB2C3EAFF0301B35104E0EE6A030154
:060E1000B307F9D7120040
:0A0E16001201000200000008D804D9
:100E20003C0001010102000109022900010100C08A
:100E30003209040000020300000009211101000131
:100E4000221D000705810340000107050103400042
:100E5000010403090434034D006900630072006F4C
:100E600000630068006900700020005400650063A2
:100E70000068006E006F006C006F00670079002052
:100E80000049006E0063002E00260348004900441C
:100E9000002000550053004200200042006F006F08
:100EA0000074006C006F0061006400650072000651
:100EB00000FF0901A10119012940150026FF007555
:100EC0000895408100190129409100C0280E280E84
:080ED000510E550E890E120BA4
:080ED8000F0EC16E81A804D0C9
:100EE000070EC16E03D002D08BEF07F0060EF66E30
:100EF000100EF76E0900F5CF00F00800F5CF01F0F5
:100F00000D0E001802E1600E011802E100EF08F07A
:100F10008BEF07F01200F26A13EE00F023EE00F000
:100F2000F86AFC6A6DA602D00DEC02F012D804003B
:100F30005EEC06F072EC06F01AD818D8060E030123
:100F4000B45D05E16D50020B02E121EC00F0EFD73A
:100F50001200140E6F6E0301B46B0301B56B030135
:100F6000B66B18EC00F08C90959012001200030103
:100F7000BA07000EBB5BBA51BB110AE1BA6B4E0E49
:100F8000BB6F060E0301B45D02E28C8012008C7010
:020F900012004D
:0E0F9200000EF36E00EE00F0080E01D8120003
:100FA000EA6002D0EE6AFCD7F350E9601200EE6A04
:020FB000FCD76C
:061000000EEF00F01200EB
:020000040030CA
:0100000024DB
:010001000EF0
:010002003FBE
:010003001EDE
:010005008179
:010006008178
:010008000FE8
:01000900C036
:01000A000FE6
:01000B00E014
:01000C000FE4
:01000D0040B2
:00000001FF
